:0200000480007A
:100000006F00C004732F2034930F8000630AFF0336
:10001000930F90006306FF03930FB0006302FF038A
:10002000170F0080130F0FFE63040F0067000F000F
:10003000732F203463540F006F00400093E19153FD
:10004000171F000023203FFC6FF09FFF930000006C
:10005000130100009301000013020000930200004E
:100060001303000093030000130400009304000036
:10007000130500009305000013060000930600001E
:100080001307000093070000130800009308000006
:100090001309000093090000130A0000930A0000EE
:1000A000130B0000930B0000130C0000930C0000D6
:1000B000130D0000930D0000130E0000930E0000BE
:1000C000130F0000930F0000732540F1631005002B
:1000D000970200009382020173905230735000180F
:1000E000970200009382020273905230B7020080A0
:1000F0009382F2FF7390023B9302F0017390023AF5
:100100007350403097020000938242017390523046
:10011000735020307350303093010000970200007C
:10012000938282EE73905230130510001315F5017F
:10013000634C05000F00F00F930110009308D005E9
:10014000130500007300000097020080938282EB89
:10015000638A020073905210B7B20000938292102B
:100160007390223073500030372500007320053023
:100170007350300097020000938242017390123452
:10018000732540F1730020309301200017250000F3
:10019000130545E78326050013052000537005D09D
:1001A00073101000530500E0631AD5069301300068
:1001B00017250000130545E5832605001305E0FF1C
:1001C000537005D073101000530500E06318D50478
:1001D0009301400017250000130545E38326050021
:1001E00013052000537015D073101000530500E064
:1001F0006316D5029301500017250000130545E151
:10020000832605001305E0FF537015D0731010000E
:10021000530500E06314D500631030020F00F00FA7
:10022000638001009391110093E111009308D005C0
:1002300013850100730000000F00F00F9301100000
:100240009308D0051305000073000000731000C070
:10025000000000000000000000000000000000009E
:10026000000000000000000000000000000000008E
:10027000000000000000000000000000000000007E
:04028000000000007A
:1010000000000000000000000000000000000000E0
:1010100000000000000000000000000000000000D0
:1010200000000000000000000000000000000000C0
:1010300000000000000000000000000000000000B0
:081040000000000000000000A8
:1020000000000040000000C0000000400000804FC1
:040000058000000077
:00000001FF
